:10000000FF2383169000831216291830A0000000E9
:10001000A00B072800349430A0006430A100000039
:10002000A00B0F28FA30A000A10B0F28000000340D
:1000300001309F000730A000A00B1C289F14073040
:10004000A000A00B21289F1823281E08A3008316B8
:100050001E088312A400003418202308A5006400A1
:10006000261C332836285430B10038287E30B100A1
:10007000640031082502031C3E28402855202C2806
:1000800000346400851841286400851C44286400FD
:1000900085184728A801A80A0520851C4B280D3083
:1000A0002802031C5428412800344630A900AA0025
:1000B0006400851C66280520A903031D58284630C6
:1000C000A900AA03031D5828782058286400851C1D
:1000D0006628640085186928A801A80A0520851CDF
:1000E0006D280D302802031C7628552888200034FE
:1000F0008820882088200B200B20902090209020A2
:100100000B200B208820882088200B200B20003417
:10011000640005150B200B200B2005110B2000346B
:10012000640005150B2005110B20003405168516FB
:100130000130AB000E30AC00003464008518AF28ED
:10014000A80A2A3028020318A8016430A9006430E4
:10015000AA000930A000A00BAB28000000346430D6
:100160002A02031DB92864302902031DBD28A903F2
:10017000D4280000000000000000A903031DCA28C5
:100180006430A900AA03031DCF286430AA0096207A
:100190007820D32800000000000000000000063096
:1001A000A000A00BD1280034B003031DED281820B7
:1001B0002308A5006400261CDE28E1284530B10094
:1001C000E3286930B100640031082502031CE928E6
:1001D000EB2896205520A801003418302802031C73
:1001E000FD2824302802031805290F30AF001630EF
:1001F0002802AB002F02AC000D290130AB000E30FD
:10020000AC000000000000000D290E30AB000130F2
:10021000AC000000000000000D29A8010000000053
:100220000000000000000000000000348316FE30D3
:1002300081000B308500831207309900831631301E
:100240009F008312A001A101A201A301A401A501A5
:10025000A601A701A801051685166430A90064301F
:10026000AA00AB01AC010130AB000E30AC00AD0117
:10027000AE01AF01B001B101B20164000F30A200C4
:1002800064000B20A20B4029640018202308A5005D
:1002900064000030A6007E302502031C5329013083
:1002A000A60090200B2090200B2090200A30A20066
:1002B00064000B20A20B58296400412005150B2077
:1002C0000B200B200B200B20051164002B03031DBA
:1002D000702905168516B203031D72292C20722978
:1002E0008512B20164002B08AD002C08AE00AD03EE
:1002F00003197D2905129D207729AE03031983294F
:0803000005169D207D296529E9
:084000000000020002000000B4
:02400E008C3FE5
:00000001FF
